:020000040000fa
:080000000205040000000000ed
:020000040000fa
:020000040002f8
:04afe000dfff00008f
:020000040000fa
:020000040002f8
:04afe400ffff00006b
:020000040000fa
:020000040002f8
:04afe80078ff0000ee
:020000040000fa
:020000040002f8
:04afec007dff0000e5
:020000040000fa
:020000040002f8
:04aff00078ff0000e6
:020000040000fa
:1000080000000000000000000000000000000000e8
:10001800fa040000000000000000000000000000da
:100028007e08000000000000000000000000000042
:10003800000000000000000000000000b2080000fe
:10004800e408000000000000000000007e09000035
:100058000000000000000000000000000000000098
:100068000000000000000000000000000000000088
:100078000000000000000000000000000000000078
:100088000000000000000000000000000000000068
:10009800140900000000000000000000000000003b
:1000a8000000000000000000000000000000000048
:1000b8000000000000000000000000000000000038
:1000c8000000000000000000000000000000000028
:1000d8000000000000000000000000000000000018
:1000e8000000000000000000000000000000000008
:1000f80000000000000000000000000000000000f8
:1001080000000000000000000000000000000000e7
:1001180000000000000000000000000000000000d7
:1001280000000000b6090000000000000000000008
:1001380000000000000000000000000000000000b7
:1001480000000000000000000000000000000000a7
:100158000000000000000000000000000000000097
:100168000000000000000000000000000000000087
:100178000000000000000000000000000000000077
:100188000000000000000000000000000000000067
:100198000000000000000000ea090000160a000044
:1001a800420a0000000000000000000000000000fb
:1001b8000000000000000000000000000000000037
:1001c8000000000000000000000000000000000027
:1001d8000000000000000000000000000000000017
:1001e8000000000000000000000000000000000007
:1001f80000000000000000000000000000000000f7
:1002080000000000000000000000000000000000e6
:1002180000000000000000000000000000000000d6
:1002280000000000000000000000000000000000c6
:1002380000000000000000000000000000000000b6
:1002480000000000000000000000000000000000a6
:100258000000000000000000000000000000000096
:100268000000000000000000000000000000000086
:0c0278000000000000000000000000007a
:020000040000fa
:10040000803e2000030007008100e900fcff3a0065
:1004100000000600831f7800c20320000400bc0017
:1004200066015100e0815900f23fb1000380b10044
:1004300006003500ee03090000000000423fb10055
:100440000380b100fbff3d001200b000223fb0006e
:10045000020035000280090000000000cf01780092
:1004600000000600040020000300370014002000f4
:100470000100370014002000889fbe008a9fbe0044
:10048000841f7800070107004f0078001100330037
:10049000f0ff2f00838f6c0006003b000405650011
:1004a0000a00a7000800370009f0a600100020008d
:1004b00008003700820f5400838f5c00030039006e
:1004c0001000200001003e000000200009f0a700fd
:1004d0000000ea004f05be004f04be000000e0002f
:1004e0000000060003f0a200869fbe00889fbe00a9
:1004f0008a9fbe008c9fbe00ea0007002c013300db
:100500006450e1004f0032006420e10052003200ec
:1005100003826c0007003b000905d0000306d000f1
:10052000820f54000c065d00020039000200320008
:1005300089017800030678008582550004003d009b
:100540000003fd008103fd008502ea008b85420067
:10055000840f720002003b0060001000e080180071
:100560006011b8000005eb007a28e1000a003900ac
:1005700006007800c75ddd00f707b20087807500d0
:100580002d003700828171000a017800610560004a
:100590008180d1000080d3008502e900f9ff3b0093
:1005a000060440008784480002003b0060041400f9
:1005b000e0841c000988a300070032008a817100d2
:1005c00082817100610164008904d1000884d30034
:1005d0008b05e800170037000978a30013003a00e4
:1005e0000b00e000130034008b05e9000804440010
:1005f00089844c000a4474000978a3000d003a0075
:100600000b00e000070034008b05e90008044400fb
:1006100089844c0001003a000b0020000978a300f7
:10062000f7ff32000001eb00020037008281710009
:100630000a017800b80007000cf0a70001f0a00044
:10064000e40037006420e10002003a00838f6c0070
:10065000e50033000801be000200be00dd003700e7
:10066000869fbe00889fbe008a9fbe008c9fbe00f2
:100670008c000700ce00330003866c006450e1005c
:100680002e0032006420e100330032006150e100ae
:100690002f0032006120e1003100320085855500d5
:1006a000eb07b00009002000080420000500370017
:1006b0000804440089844c000a003100060343000a
:1006c00087834b000001530081815b00f8ff3300fa
:1006d0000203be000800a0000804440089844c0006
:1006e000f6ff3900c639dd008301730001003200d6
:1006f000130020008904d1000884d3000998a300c6
:10070000050032000800a7000300a0008904d10002
:100710000884d3008b05e8008904d1000884d30045
:100720000001eb000281d2007b00070001f0a10074
:100730000cf0a70001f0a000a60037006420e10043
:10074000a90032000801be000200be00f7ff37001a
:100750006120e100a40032006000b800f3ff370020
:100760000000200001f82700f0ff3700829fbe0044
:100770000001be00530007000470a70003f0a100b1
:1007800003f8a30015003a006509b100110032001a
:100790000a0035006928e100030035000100280047
:1007a0004f01be00000005000000400081804800ad
:1007b0008502e900fcff3a0006003700f88f42008e
:1007c000060035008100d1000080d3008502e800da
:1007d000fcff3a004f01be00000006008000eb0065
:1007e0004f01be00000005000080fb008000eb0010
:1007f000829fbe00889fbe008a9fbe0001057800d0
:100800000100e0000400350008003c000000e000aa
:10081000200032000500370060001000e080180062
:1008200002003b0001f024001a0037000004be0063
:100830006011b8006b0920000982cf000200390066
:100840000882cf000441b000694252000e0032001d
:1008500008003b0082817100610164008904d100bd
:100860000884d3008b05e8000442e800f9ff3a0051
:10087000050037000804440089844c008b05e9001a
:100880000442e900fbff3a00230007000af0a7003a
:1008900001f0a0004f05be004f04be004f01be0096
:1008a000000006000004be00060007000003be00b2
:1008b0000405be000200be0002000700844f750060
:1008c00000000600c70ade00f107b200f50fb20013
:1008d00008003200e1cf4200020032000170a000a7
:1008e00024000500810f700001003200040805009b
:1008f00044000500810f700002003a00140005005a
:100900008502e9000000400081c04800fcff3b0078
:100910000170a000240005008100200061805500c6
:100920000b003d000b00200061fe2f000100e100e4
:100930001d00340082817100610164008904d100ce
:100940000884d3000000e800faff3a00710020009c
:1009500061006400030070000200600009003200c2
:1009600061044400e0844c000988a50005003200c1
:100970008b05e8006808e10002003a008904d10014
:100980000884d300f20f20000258e10005003d006a
:10099000c75ddd00f907b2008980750008007800a6
:1009a000000006000bf827008b007800000005000f
:1009b0000200be006450e100050036006420e10042
:1009c000020036000968a30001003a000800be00da
:1009d0000160a0004f06be004f05be004f04be00e0
:1009e0004f03be0000000600f0ff2f00f1ff2700bc
:1009f000f8ff37000020ef000220ef00c088a900b8
:100a0000004006000f00210090272100000188000f
:100a1000000000000000eb00000778000c00090057
:100a2000002f78000007eb005420ef000e2eef009f
:100a30001e2eef000000eb00e11c2100311e09001a
:100a40008018780040a7a900a10020006cfe0700d4
:100a5000e0022000303a880044e7a90044c7a9001a
:100a60004407a9004427a9004447a9004467a900f6
:100a70004487a900300020000600fc0031742000eb
:100a800082072000a309200082487800834878006c
:100a900080487800113a8000618070000600fc00f8
:100aa0002174200062042000730520008248780031
:100ab00083487800804878004427ef00e002200057
:100ac000303a8800300020000d00fc003174200016
:100ad00082072000a309200082487800834878001c
:100ae000804878000000200021742000620420006b
:100af0007305200082487800834878008048780099
:100b000042a7ae00feff3700813e20003cfe0700fa
:100b100010c0b30086e6b70090c2b300c4e6b700c9
:100b20000002200000708800007825008070880096
:100b300010aea90010cea9004008a9004028a900c5
:100b40004048a9000008a9002008a9004188a90080
:100b500041a8a90041c8a9002068a90011a1a900c5
:100b60001061a9001021a90010a1a8001081a800ff
:100b70000621ef00008020006008880000e8a9003e
:100b80004388a80043a8a90043c8a80020e8a800fb
:100b900011e1a90013a1a90013e1a8001221a900e5
:100ba00012a1a8001281a8004408a8004428a900a6
:100bb0004448a9000a21ef000ea1ef000108a90096
:100bc0002108a80013e1a8004d88a9004da8a9009c
:100bd0004dc8a9000368a9002368a90021e1a80065
:100be00021a1a90020c1a90020a1a8002081a8005e
:100bf0002021a9001821ef00402e2200e0088800e3
:100c00004e08a9004e28a9004e48a8000388a90054
:100c10002388a8002002a9002022a9002042a900c0
:100c200020a2a9002062a9002082a90020e2a90038
:100c30002102a9002122a90070072000401188008c
:100c400022a2a90022c2a90022e2a90021e2a80052
:100c50002182a9004588a90045a8a80045c8a80088
:100c60002168a8002828a8002bc8a9002be8a90003
:100c70002c08a9000bc8a9000be8a9000c08a900c2
:100c800001eca90001aca900016ca900014ca8006d
:100c9000012ca900010ca90000eca900008ca900fe
:100ca00000aca90000cca900000ca900002ca900f0
:100cb000004ca900006ca900202cef00402cef0094
:100cc000602cef0020eca800200ca80040eca8004d
:100cd000400ca80060eca800600ca800f07f200089
:100ce00020608800020ca900022ca900024ca90077
:100cf0000040200030618800462cef00662cef0099
:100d0000282cef00482cef00682cef000aacef0015
:100d100023eca80023cca80043eca80043cca900f6
:100d200063eca80063cca90023aca900238ca90024
:100d3000dabc2a001b32240030002c00fa60880044
:100d4000fb60880020618800dabc2a001b32240086
:100d500020002c00fa608800fb6088001061880089
:100d6000dabc2a001b32240030002c00fa60880014
:100d7000fb60880020628800dabc2a001b32240055
:100d800000002800fa608800fb608800106288007c
:100d9000dabc2a001b32240030002c00fa608800e4
:100da000fb60880020638800dabc2a001b32240024
:100db00000002800fa608800fb608800106388004b
:100dc000a70037003f0037000020200000618800a6
:100dd00000202000006288000020200000638800be
:100de000020ca900022ca800024ca80004acef00e1
:100df00028acef0048acef0068acef00262cef0009
:100e0000462cef00662cef000aacef0023eca800a4
:100e100023cca90043eca80043cca90063eca800b4
:100e200063cca900dabc2a001b32240030002c005d
:100e3000fa608800fb60880020618800dabc2a0024
:100e40001b32240000002800fa608800fb60880044
:100e500010618800dabc2a001b32240030002c000c
:100e6000fa608800fb60880020628800dabc2a00f3
:100e70001b32240000002800fa608800fb60880014
:100e800010628800dabc2a001b32240030002c00db
:100e9000fa608800fb60880020638800dabc2a00c2
:100ea0001b32240000002800fa608800fb608800e4
:100eb0001063880011eea90011aea900116ea900ff
:100ec00067003700350037000010200000618800ff
:100ed00000102000006288000010200000638800dd
:100ee000020ca900022ca800024ca8000a2cef005a
:100ef00004acef00282cef0050552500406288001c
:100f0000a0aa2a0040638800dabc2a001b32240011
:100f100030002c00fa608800fb60880020618800a7
:100f2000dabc2a001b32240000002c00fa60880082
:100f3000fb60880010618800dabc2a001b322400a4
:100f400030002c00fa608800fb6088002062880076
:100f5000dabc2a001b32240000002c00fa60880052
:100f6000fb60880010628800dabc2a001b32240073
:100f700030002c00fa608800fb6088002063880045
:100f8000dabc2a001b32240000002c00fa60880022
:100f9000fb608800106388003100370030003700a4
:100fa000001020000061880000102000006288000e
:100fb000020ca900022ca800024ca8000a2cef0089
:100fc00004acef00282cef000000240040628800f1
:100fd000dabc2a001b32240030002c00fa608800a2
:100fe000fb60880020618800dabc2a001b322400e4
:100ff00000002c00fa608800fb6088001061880007
:10100000dabc2a001b32240030002c00fa60880071
:10101000fb60880020628800dabc2a001b322400b2
:1010200000002c00fa608800fb60880010628800d5
:10103000dabc2a001b32240030002c00fa60880041
:10104000fb60880020638800dabc2a001b32240081
:1010500000002c00fa608800fb60880010638800a4
:10106000218ca900418ca900618ca900216ca900e8
:10107000416ca900616ca900214ca900414ca90058
:10108000614ca90020eca80040eca80060eca8008e
:101090003e2cef005e2cef007e2cef0001eca80050
:1010a0000000eb00e1412100ff00090080587800ba
:1010b000ff71ef000072ef00f603070020c0b300dd
:1010c000e0f1b70020c0b300e1f1b700f10607007e
:1010d0001672ef0000142000b08e8800e231ef009d
:1010e000e431ef00ee31ef00f031ef0010cea90057
:1010f00014cea8009303070004013700ff3ffc0053
:101100004200f8003600f8004400f8008e1f780016
:101110000e0020000d000900be1f78003200f8000c
:101120000100fc000008a9002068a9000068a900cf
:101130000040200030618800ff3ffc003200f900d1
:10114000ae0120000d0009004f1778004f0778000e
:101150004400f9003600f9004200f9000100fc00eb
:1011600000400600ff3ffc004200f8003600f80097
:101170004400f8008e1f78000e0020000d000900ca
:10118000be1f78003200f8000100fc0000e8a90052
:10119000b08e800060088800e231ec00ff3ffc0068
:1011a0003200f900ae0120000d0009004f17780051
:1011b0004f0778004400f9003600f9004200f900ba
:1011c0000100fc0000400600ff3ffc004200f80068
:1011d0003600f8004400f8008e1f78000e00200052
:1011e0000d000900be1f78003200f8000100fc006d
:1011f0000108a900128eaa00108ea900ff3ffc0072
:101200003200f900ae0120000d0009004f177800f0
:101210004f0778004400f9003600f9004200f90059
:101220000100fc0000400600ff3ffc004200f80007
:101230003600f8004400f8008e1f78000e002000f1
:101240000d000900be1f78003200f8000100fc000c
:101250000388a9001732ae00110037001c72ec00a1
:101260001c12ae00070037001bd2bf000080fb003d
:1012700000004000e1312100608078003063880088
:10128000060037001ad2bf000080fb0000004000bb
:10129000e13121006080780030638800060037006b
:1012a0001c72ef00f28e800002014100e03121004b
:1012b000600079003063880019d2bf000080fb0015
:1012c00000004000e121210060807800e0088800f3
:1012d000ff3ffc003200f900ae0120000d000900c4
:1012e0004f1778004f0778004400f9003600f900e6
:1012f0004200f9000100fc0000400600ff3ffc0036
:101300004200f8003600f8004400f8008e1f780014
:101310000e0020000d000900be1f78003200f8000a
:101320000100fc000168a900ff71ec00ffd1bf00c3
:101330008080fb0030118000e24121008070790044
:10134000ff3ffc003200f900ae0120000d00090053
:101350004f1778004f0778004400f9003600f90075
:101360004200f9000100fc0000400600ff3ffc00c5
:101370004200f8003600f8004400f8008e1f7800a4
:101380000e0020000d000900be1f78003200f8009a
:101390000100fc000828a9002242ae00000037002e
:1013a0002222af002222a900ff3ffc003200f900f8
:1013b000ae0120000d0009004f1778004f0778009c
:1013c0004400f9003600f9004200f9000100fc0079
:1013d00000400600ff3ffc004200f8003600f80025
:1013e0004400f8008e1f78000e0020000d00090058
:1013f000be1f78003200f8000100fc000bc8a900f5
:10140000ff3ffc003200f900ae0120000d00090092
:101410004f1778004f0778004400f9003600f900b4
:101420004200f9000100fc0000400600ff3ffc0004
:101430004200f8003600f8004400f8008e1f7800e3
:101440000e0020000d000900be1f78003200f800d9
:101450000100fc000be8a900ff3ffc003200f9008e
:10146000ae0120000d0009004f1778004f077800eb
:101470004400f9003600f9004200f9000100fc00c8
:1014800000400600ff3ffc004200f8003600f80074
:101490004400f8008e1f78000e0020000d000900a7
:1014a000be1f78003200f8000100fc000c08a90003
:1014b000ff3ffc003200f900ae0120000d000900e2
:1014c0004f1778004f0778004400f9003600f90004
:1014d0004200f9000100fc000040060000d2bf00fd
:1014e000ff51e300070032000072ec0000d2bf00a1
:1014f0000080fb00e141210060c0780001f2b700ec
:101500000100370001f2ef0000000600f3ff0700c2
:1015100040cbb3000152b50006003900e0cfb30064
:101520000152b50001003900010037000272ef00de
:10153000c600370001f2ae00370037000272ef003c
:1015400030c8b3000152e30005003a0001d2bf00e9
:1015500002f2b70003f2ef0004f2ef002d003700b3
:1015600030c9b3000152e30005003a0001d2bf00c8
:1015700002f2b70005f2ef0006f2ef002500370097
:1015800030cab3000152e30005003a0001d2bf00a7
:1015900002f2b70007f2ef0008f2ef001d0037007b
:1015a00030cbb3000152e30005003a0001d2bf0086
:1015b00002f2b70009f2ef000af2ef00150037005f
:1015c00030ccb3000152e30004003a0001d2bf0066
:1015d00002f2b7000bf2ef000e00370030cdb3007f
:1015e0000152e30004003a0001d2bf0002f2b7004a
:1015f0000cf2ef000700370030ceb3000152e300d9
:1016000004003a0001d2bf0002f2b7000df2ef0071
:101610000ef2ef008d0037000252e20002003a00a5
:101620008a0037008900370030c8b3000252e30057
:101630001f003a0000e0ef000352e30003003a000d
:1016400001d2bf0003f2b700180037000152ec00ce
:1016500004f2b70003d2bf001152b50012003a00e5
:101660001672ef00e08e800060fc0700708f88002b
:10167000818f880004d2bf005bfc07000001be0020
:10168000e08e800059fc0700f5fb0700d08f880032
:10169000e18f88001652a800e231ef00e431ef003c
:1016a00011e1a8001732a90003f2ef00670037002c
:1016b00030c9b3000252e3004b003a0000e0ef00f3
:1016c0000552e30003003a0001d2bf0005f2b70063
:1016d0004400370001d2bf0006f2b7000652e20014
:1016e00016003a0005d2bf001152b50012003a00b0
:1016f0001672ef00e08e80003cfc0700708f8800bf
:10170000818f880015d2bf0037fc07000001be00a2
:10171000e08e800035fc0700d1fb0700d08f8800e9
:10172000e18f88001652a800e231ef00e431ef00ab
:1017300011e1a8001732a9002a00370080c1b300c8
:101740000552b5000100310025003700b0c5b300d7
:101750000552b500010039002100370005d2bf0055
:1017600011f2b70006d2bf000080fb00e08e8800b7
:10177000d18e800006d2bf000080fb000100400037
:10178000c08e8800c18e8000f0072000808f50003e
:1017900002003600f0072000c08e88001672ef00ad
:1017a000ee31ef00f031ef00462cef001612a800ea
:1017b00013d2bf000cfc07000001be00c08e8000e9
:1017c0000afc0700a6fb0700908f8800a18f880005
:1017d000e231ef00e431ef0011e1a80014cea800df
:1017e00005f2ef001900370030cab3000252e300df
:1017f0000a003a0000e0ef000752e30003003a005d
:1018000001d2bf0007f2b7000300370001d2bf00ca
:1018100008f2b700e80007000c00370030cbb30037
:101820000252e30009003a0000e0ef000952e30031
:1018300003003a0001d2bf0009f2b70003003700ed
:1018400001d2bf000af2b700e1000700218f80003b
:10185000108f8000808f5000bf003100e431ec0019
:1018600016d2bf0080407800e1cf50004a003a0015
:10187000c08e8000ddfb07000001be00708f80007d
:10188000818f8000f9fa070042003c00728f8000cf
:10189000838f8000908f8000a18f800012fb070053
:1018a000708f8800818f8800728f8000838f800006
:1018b000c08e8000cdfb0700eefa07002b003d0034
:1018c000c08e8000c9fb0700708f8800818f880060
:1018d000c28e800002014100e031210060007900e9
:1018e00030628800c08e8000dc11b500bffb0700ad
:1018f000b08f8800c18f880014d2bf00bafb0700e8
:101900000001be00b08f8000c18f800054fb070033
:10191000b08f8800c18f88006011b800b08f800040
:10192000c18f8000cffa070008003a00e28e8000e5
:1019300002014100e031210060007900306288003e
:101940001672ef0011e1a900060037001612a90077
:101950001632a800e231ef00e431ef0011e1ae00f1
:1019600011e1a8001732a8000a003700708f80002c
:10197000818f80007dfb070010f2b70010d2bf00fe
:101980000080fb0000004000e13121006080780011
:10199000306288007000370016d2bf0080407800a7
:1019a000e2cf500046003a00728f8000838f8000a3
:1019b000b08f8000c18f8000cbfa0700708f880045
:1019c000818f8800f1f1ae0002003700ee31ef00a8
:1019d000f031ef00f9f1ae001b003700728f80008c
:1019e000838f8000e08e800080fb0700a1fa070053
:1019f0000d003d00708f8000818f80005bfb070031
:101a000010f2b70010d2bf000080fb0000004000c1
:101a1000e1312100608078003062880011e1ae0081
:101a200011e1a80007003700e28e800002014100aa
:101a3000e031210060007900306288001672ef000a
:101a400011e1a9001d003700f9f1af001b003700bc
:101a5000e08e800065fb07000001be00708f8000f3
:101a6000818f800083fa07000d003d00708f800099
:101a7000818f80003dfb070010f2b70010d2bf003d
:101a80000080fb0000004000e13121006080780010
:101a90003062880011e1ae0011e1a80007003700b4
:101aa000e28e800002014100e031210060007900f7
:101ab000306288001672ef0011e1a900260037009d
:101ac00016d2bf0080407800e4cf500022003a00d8
:101ad000708f8000818f8000d28f8000e38f800024
:101ae00080fa0700708f8800818f88000200200034
:101af00003002000708f8000818f80005bfa070058
:101b000006003c001672ef00462cef001172ef0049
:101b100014cea90011e1a9000f003700708f8000da
:101b2000818f800011fb070010f2b70010d2bf00b8
:101b30000080fb0000004000e1312100608078005f
:101b40003062880011e1af0003003700e231ef009e
:101b5000e431ef0011e1a8001612af00040ea80056
:101b60001612ae00040ea9001632af00042ea80013
:101b70001632ae00042ea9001652af00142ea80093
:101b80001652ae00142ea9001652e20006003a00ca
:101b90001152e20002003600140ea80001003700c6
:101ba000140ea90001003700140ea90012aeaa00fd
:101bb00010aea90055fe370007f2ef000000060046
:101bc0000bf2ef00000006000cf2ef000000060030
:101bd00009d2bf0080407800e5cf500026003a00cf
:101be0000ad2bf0018f2b7001872d5001852e200ee
:101bf00008003a000388a9002388a900f28e80001b
:101c000002014100e031210060007900306388006a
:101c100018003700f18e800018d2bf000080fb0052
:101c2000810f5000020036001a72ef0003003700e7
:101c300018d2bf00de51b5001af2b700f18e800055
:101c400018d2bf000080fb00010040008000780037
:101c5000f0072000808f500003003600f0c7b3006b
:101c60001bf2b70003003700f08e80001852b4005a
:101c70001bf2b700aa00370009d2bf0080407800ed
:101c8000e6cf500016003a000ad2bf0019f2b700a2
:101c90000a52e2000a0036001821ef000388a9006a
:101ca00019d2bf000080fb0000004000e1212100ac
:101cb00060807800e00888002388a80007003700cb
:101cc0000388a9002388a900f28e80000201410048
:101cd000e031210060007900306388009000370017
:101ce00009d2bf0080407800e7cf500022003a00c0
:101cf0000ad2bf000080fb00f08e8800f18e8000c9
:101d000018d2bf000080fb00810f50000200360097
:101d10001a72ef000300370018d2bf00de51b50081
:101d20001af2b700f18e800018d2bf000080fb00cd
:101d30000100400080007800f0072000808f5000f4
:101d400003003600f0c7b3001bf2b70003003700f2
:101d5000f08e80001852b4001bf2b7000ad2bf0008
:101d60000080fb0000004000e1312100608078002d
:101d7000306388006a00370009d2bf0080407800d5
:101d8000efcf500008003a000ad2bf0012f2b700ad
:101d900012d2bf000080fb000020ec004400dd00f8
:101da000b08e88005e00370009d2bf008040780006
:101db000f0cf500003003a000a52ec0013f2b700d3
:101dc0005700370009d2bf0080407800f1cf5000a3
:101dd00005003a000ad2bf000080fb000020ec00a2
:101de000d08e88004e00370009d2bf0080407800b6
:101df000f2cf500003003a000a52ec0014f2b70090
:101e00004700370009d2bf0080407800f3cf500070
:101e100003003a000a52ec0015f2b7004000370008
:101e200020c4b3000952e30007003a000a52e2005e
:101e300002003a003c00070002003700048ea800b0
:101e4000650007003600370000c5b3000952e30003
:101e50002a003a000a52ec00e0f1b700e0d1bf00de
:101e60000080fb004500de00e0f1b700e1d1bf00db
:101e7000e051e3002000320014cea800462cef0011
:101e80001172ef00e051e20002003a008105070004
:101e900017003700e0d1bf0080407800e1cf50004c
:101ea00002003a007b04070011003700e0d1bf00b8
:101eb00080407800e2cf500002003a00750307002e
:101ec0000b003700e0d1bf0080407800e3cf500026
:101ed00002003a006f02070005003700e0d1bf00a2
:101ee00080407800e4cf500001003a00690107000b
:101ef000e0d1bf00e1f1b70009003700b0c7b3007f
:101f00000952e30006003a00462cef001672ef007b
:101f100014cea8001732a9001172ef000ff2ef00e3
:101f200009f2ef0000000600462cef00662cef00df
:101f30001672ef0014cea800008ea900048ea9002e
:101f40000000370000062000f08e8800f28e80002e
:101f500002014100e0312100600079003063880017
:101f600014cea80040c0b30018f2b70040c1b300bf
:101f700019f2b7001800070040c1b30012f2b70011
:101f800012d2bf000080fb000020ec004400dd0006
:101f9000b08e880040c2b30013f2b70040062000a4
:101fa000d08e880000c2b30014f2b70000c5b300a1
:101fb00015f2b70020c0b300e051b50005003200b3
:101fc0003403070020c0b300e0f1b70020c0b30025
:101fd000e1f1b7000000060018d2bf008080fb00ce
:101fe00019d2bf000080fb000200bc000200e0002c
:101ff00022003600f18e800018d2bf000080fb0066
:10200000810f5000020036001a72ef000300370003
:1020100018d2bf00de51b5001af2b700f18e800071
:1020200018d2bf000080fb00010040008000780053
:10203000f0072000808f500003003600f0c7b30087
:102040001bf2b70003003700f08e80001852b40076
:102050001bf2b7001821ef000388a90019d2bf00b6
:102060000080fb0000004000e1212100608078003a
:10207000e00888002388a80005003700f28e800061
:1020800002014100e03121006000790030638800e6
:10209000000006001eb2ef00a0c7250000918800d6
:1020a00050982500109188004081250020918800db
:1020b000906a2500309188003054250040918800b6
:1020c000303e2500509188009028250060918800be
:1020d000501325007091880060fe240080918800d4
:1020e000c0e924009091880080d52400a091880048
:1020f00090c12400b0918800f0ad2400c091880008
:10210000a09a2400d0918800a0872400e091880044
:10211000f0742400f09188009062240000928800fe
:102120008050240010928800b03e24002092880045
:10213000302d240030928800f01b2400409288004b
:10214000000b24005092880050fa2300609288000f
:10215000e0e9230070928800c0d9230080928800b3
:10216000e0c923009092880040ba2300a092880022
:10217000e0aa2300b0928800c09b2300c092880090
:10218000e08c2300d0928800307e2300e09288000b
:10219000d06f2300f0928800a06123000093880094
:1021a000b053230010938800f0452300209388004b
:1021b0007038230030938800202b23004093880040
:1021c000101e230050938800401123006093880064
:1021d000900423007093880020f8220080938800e8
:1021e000e0eb220090938800d0df2200a0938800cb
:1021f000f0d32200b093880050c82200c09388001a
:10220000d0bc2200d093880080b12200e0938800e7
:1022100070a62200f0938800809b22000094880022
:10222000c09022001094880020862200209488000c
:10223000c07b220030948800807122004094880086
:102240006067220050948800805d220060948800be
:10225000c053220070948800204a22008094880095
:10226000b04022009094880060372200a09488003b
:10227000402e2200b094880040252200c09488009f
:10228000601c2200d0948800b0132200e0948800e3
:10229000200b2200f0948800b002220000958800f4
:1022a00060fa21001095880040f2210020958800f6
:1022b00030ea21003095880050e2210040958800e6
:1022c00090da210050958800e0d2210060958800c6
:1022d00060cb210070958800f0c3210080958800b4
:1022e000b0bc21009095880080b52100a0958800a1
:1022f00080ae2100b095880090a72100c09588008d
:10230000b0a02100d0958800009a2100e0958800b7
:1023100060932100f0958800e08c210000968800f1
:102320008086210010968800308021002096880049
:10233000007a210030968800f073210040968800d2
:10234000f06d21005096880000682100609688009a
:102350004062210070968800805c21008096880091
:10236000e05621009096880060512100a0968800d8
:10237000f04b2100b096880090462100c09688005e
:1023800050412100d0968800203c2100e096880032
:1023900010372100f0968800103221000097880045
:1023a000202d2100109788004028210020978800c8
:1023b0008023210030978800d01e2100409788009c
:1023c000301a210050978800a015210060978800de
:1023d0002011210070978800c00c21008097880090
:1023e000700821009097880020042100a0978800a1
:1023f000f0ff2000b0978800d0fb2000c097880035
:10240000c0f72000d0978800d0f32000e097880024
:10241000e0ef2000f097880000ec20000098880092
:1024200030e820001098880070e420002098880090
:10243000c0e020003098880020dd2000409888000f
:1024400090d920005098880010d62000609888000d
:10245000a0d220007098880040cf2000809888008b
:10246000e0cb200090988800a0c82000a0988800a9
:1024700060c52000b098880030c22000c098880055
:1024800010bf2000d098880000bc2000e098880091
:10249000000006001e33ef001000200000998800a5
:1024a000200020001099880030002000209988002a
:1024b00030002000309988003000200040998800ca
:1024c000300020005099880030002000609988007a
:1024d000300020007099880040002000809988001a
:1024e000400020009099880040002000a0998800ba
:1024f00040002000b099880040002000c09988006a
:1025000050002000d099880050002000e0998800f9
:1025100050002000f099880050002000009a8800a8
:1025200060002000109a880060002000209a880037
:1025300060002000309a880070002000409a8800d7
:1025400070002000509a880070002000609a880077
:1025500080002000709a880080002000809a880007
:1025600090002000909a880090002000a09a880097
:10257000a0002000b09a8800a0002000c09a880027
:10258000b0002000d09a8800c0002000e09a8800a7
:10259000c0002000f09a8800d0002000009b880036
:1025a000e0002000109b8800e0002000209b8800b5
:1025b000f0002000309b880000012000409b880034
:1025c00010012000509b880020012000609b8800a3
:1025d00030012000709b880040012000809b880013
:1025e00050012000909b880060012000a09b880083
:1025f00070012000b09b880090012000c09b8800e3
:10260000a0012000d09b8800b0012000e09b880042
:10261000d0012000f09b8800e0012000009c880091
:1026200000022000109c880020022000209c8800ce
:1026300040022000309c880060022000409c8800fe
:1026400080022000509c8800a0022000609c88002e
:10265000c0022000709c8800f0022000809c88004e
:1026600010032000909c880040032000a09c88005c
:1026700070032000b09c8800a0032000c09c88004c
:10268000d0032000d09c880010042000e09c88002b
:1026900040042000f09c880080042000009d8800f9
:1026a000c0042000109d880000052000209d8800a7
:1026b00050052000309d8800a0052000409d880026
:1026c000e0052000509d880040062000609d8800a5
:1026d00090062000709d8800f0062000809d8800f4
:1026e00050072000909d8800c0072000a09d880012
:1026f00030082000b09d8800a0082000c09d880000
:1027000020092000d09d8800a0092000e09d8800bd
:10271000200a2000f09d8800b00a2000009e88005a
:10272000500b2000109e8800f00b2000209e880097
:10273000900c2000309e8800400d2000409e8800b4
:10274000000e2000509e8800c00e2000609e880071
:10275000a00f2000709e880070102000809e8800ce
:1027600060112000909e880050122000a09e8800da
:1027700060132000b09e880070142000c09e880066
:1027800090152000d09e8800c0162000e09e880092
:1027900000182000f09e880060192000009f88002b
:1027a000c01a2000109f8800401c2000209f880035
:1027b000d01d2000309f8800701f2000409f88009f
:1027c00030212000509f880010232000609f880047
:1027d00000252000709f880010272000809f88001f
:1027e00030292000909f8800802b2000a09f880027
:1027f000f02d2000b09f880070302000c09f88001e
:1028000020332000d09f880000362000e09f880001
:1028100000392000f09f8800203c200000a08800a4
:10282000703f200010a088000043200020a08800f6
:10283000b046200030a08800a04a200040a08800b8
:10284000c04e200050a088002053200060a08800c7
:10285000c057200070a08800a05c200080a08800e5
:10286000c061200090a0880020672000a0a0880000
:10287000e06c2000b0a08800e0722000c0a08800ba
:1028800040792000d0a08800f07f2000e0a08800e0
:10289000000006001e33ef00600020000099880051
:1028a0007000200010998800800020002099880086
:1028b0008000200030998800800020004099880026
:1028c00090002000509988009000200060998800b6
:1028d000a000200070998800a00020008099880046
:1028e000b000200090998800b0002000a0998800d6
:1028f000c0002000b0998800c0002000c099880066
:10290000d0002000d0998800d0002000e0998800f5
:10291000e0002000f0998800f0002000009a880074
:10292000f0002000109a880000012000209a880002
:1029300010012000309a880010012000409a880081
:1029400020012000509a880030012000609a880001
:1029500040012000709a880050012000809a880071
:1029600060012000909a880070012000a09a8800e1
:1029700080012000b09a880090012000c09a880051
:10298000a0012000d09a8800b0012000e09a8800c1
:10299000d0012000f09a8800e0012000009b880010
:1029a000f0012000109b880010022000209b88006e
:1029b00020022000309b880040022000409b8800bd
:1029c00050022000509b880070022000609b88000d
:1029d00090022000709b8800b0022000809b88003d
:1029e000d0022000909b8800f0022000a09b88006d
:1029f00010032000b09b880030032000c09b88009b
:102a000060032000d09b880080032000e09b8800aa
:102a1000b0032000f09b8800d0032000009c8800b9
:102a200000042000109c880030042000209c8800b6
:102a300060042000309c880090042000409c8800a6
:102a4000d0042000509c880000052000609c880075
:102a500040052000709c880080052000809c880034
:102a6000c0052000909c880000062000a09c8800e3
:102a700050062000b09c880090062000c09c880072
:102a8000e0062000d09c880030072000e09c8800f1
:102a900080072000f09c8800e0072000009d88004f
:102aa00040082000109d8800a0082000209d88007c
:102ab00000092000309d880070092000409d88009a
:102ac000e0092000509d8800500a2000609d880089
:102ad000d00a2000709d8800500b2000809d880047
:102ae000d00b2000909d8800600c2000a09d8800e5
:102af000f00c2000b09d8800800d2000c09d880053
:102b0000200e2000d09d8800c00e2000e09d88008f
:102b1000700f2000f09d880030102000009e88007b
:102b2000f0102000109e8800b0112000209e880028
:102b300080122000309e880060132000409e880094
:102b400040142000509e880030152000609e8800b0
:102b500020162000709e880030172000809e88007c
:102b600040182000909e880060192000a09e8800d8
:102b7000801a2000b09e8800c01b2000c09e8800e4
:102b8000001d2000d09e8800601e2000e09e88006e
:102b9000c01f2000f09e880030212000009f880088
:102ba000c0222000109f880050242000209f880011
:102bb00000262000309f8800c0272000409f88000a
:102bc00090292000509f8800802b2000609f880063
:102bd000802d2000709f8800902f2000809f88000b
:102be000c0312000909f880010342000a09f8800f2
:102bf00070362000b09f880000392000c09f8800f8
:102c0000903b2000d09f8800503e2000e09f88002d
:102c100030412000f09f88003044200000a0880050
:102c20005047200010a08800a04a200020a0880063
:102c3000104e200030a08800a051200040a0880045
:102c40006055200050a088005059200060a08800e6
:102c5000705d200070a08800c061200080a0880006
:102c60004066200090a08800f06a2000a0a08800a4
:102c7000e06f2000b0a0880000752000c0a0880090
:102c8000607a2000d0a08800f07f2000e0a08800bb
:102c9000000006001e33ef0050012000009988005c
:102ca0007001200010998800800120002099880080
:102cb0009001200030998800900120004099880000
:102cc000a001200050998800b00120006099880080
:102cd000c001200070998800d001200080998800f0
:102ce000e00120009099880000022000a09988004f
:102cf00010022000b099880020022000c0998800ae
:102d000030022000d099880040022000e09988001d
:102d100060022000f099880070022000009a88006c
:102d200090022000109a8800a0022000209a8800bb
:102d3000c0022000309a8800d0022000409a88000b
:102d4000f0022000509a880010032000609a88004a
:102d500020032000709a880040032000809a880099
:102d600060032000909a880080032000a09a8800c9
:102d7000a0032000b09a8800c0032000c09a8800f9
:102d8000e0032000d09a880010042000e09a880018
:102d900030042000f09a880060042000009b880026
:102da00080042000109b8800b0042000209b880035
:102db000e0042000309b880000052000409b880034
:102dc00030052000509b880060052000609b880033
:102dd000a0052000709b8800d0052000809b880003
:102de00000062000909b880040062000a09b8800e1
:102df00070062000b09b8800b0062000c09b8800b1
:102e0000f0062000d09b880030072000e09b88005f
:102e100070072000f09b8800c0072000009c8800fd
:102e200000082000109c880050082000209c88008a
:102e3000a0082000309c8800f0082000409c8800fa
:102e400040092000509c8800a0092000609c880058
:102e5000f0092000709c8800500a2000809c8800a7
:102e6000b00a2000909c8800100b2000a09c8800d5
:102e7000800b2000b09c8800f00b2000c09c8800d4
:102e8000600c2000d09c8800d00c2000e09c8800c2
:102e9000400d2000f09c8800c00d2000009d88009f
:102ea000400e2000109d8800c00e2000209d88004c
:102eb000500f2000309d8800e00f2000409d8800ca
:102ec00070102000509d880010112000609d880027
:102ed000b0112000709d880050122000809d880055
:102ee00000132000909d8800b0132000a09d880052
:102ef00070142000b09d880030152000c09d88000f
:102f0000f0152000d09d8800c0162000e09d8800ac
:102f1000a0172000f09d880070182000009e8800f7
:102f200060192000109e8800501a2000209e880002
:102f3000401b2000309e8800401c2000409e8800de
:102f4000401d2000509e8800601e2000609e88006a
:102f5000701f2000709e8800a0202000809e8800a6
:102f6000d0212000909e880010232000a09e880081
:102f700050242000b09e8800b0252000c09e88000c
:102f800010272000d09e880080282000e09e880026
:102f9000f0292000f09e8800802b2000009f8800f0
:102fa000102d2000109f8800c02e2000209f880038
:102fb00070302000309f880040322000409f880001
:102fc00010342000509f880000362000609f880049
:102fd000f0372000709f8800003a2000809f880012
:102fe000203c2000909f8800503e2000a09f880039
:102ff000a0402000b09f880000432000c09f8800b0
:1030000070452000d09f880000482000e09f880085
:10301000a04a2000f09f8800604d200000a088009a
:103020003050200010a088002053200020a08800ed
:103030003056200030a088005059200040a0880061
:10304000a05c200050a088000060200060a08800e4
:103050008063200070a088002067200080a0880086
:10306000f06a200090a08800d06e2000a0a0880008
:10307000e0722000b0a0880020772000c0a0880067
:10308000807b2000d0a08800f07f2000e0a0880096
:10309000000006001e33ef00400420000099880065
:1030a0006004200010998800800420002099880086
:1030b000a004200030998800c004200040998800b6
:1030c000e0042000509988000005200060998800e5
:1030d00030052000709988005005200080998800f4
:1030e0007005200090998800a0052000a099880014
:1030f000c0052000b0998800e0052000c099880034
:1031000010062000d099880040062000e099880031
:1031100060062000f099880090062000009a880040
:10312000c0062000109a8800f0062000209a88002f
:1031300020072000309a880050072000409a88001d
:1031400080072000509a8800c0072000609a8800fd
:10315000f0072000709a880030082000809a8800cc
:1031600060082000909a8800a0082000a09a88009b
:10317000e0082000b09a880020092000c09a88004a
:1031800050092000d09a8800a0092000e09a880009
:10319000e0092000f09a8800200a2000009b8800a7
:1031a000700a2000109b8800b00a2000209b880035
:1031b000000b2000309b8800500b2000409b8800b3
:1031c000a00b2000509b8800f00b2000609b880023
:1031d000400c2000709b8800900c2000809b880091
:1031e000f00c2000909b8800400d2000a09b8800e0
:1031f000a00d2000b09b8800000e2000c09b88001e
:10320000600e2000d09b8800c00e2000e09b88004c
:10321000300f2000f09b8800a00f2000009c880049
:1032200000102000109c880070102000209c880056
:10323000f0102000309c880060112000409c880025
:10324000e0112000509c880050122000609c8800f3
:10325000e0122000709c880060132000809c880091
:10326000e0132000909c880070142000a09c88002f
:1032700000152000b09c880090152000c09c88009c
:1032800020162000d09c8800c0162000e09c8800fa
:1032900060172000f09c880000182000009d880026
:1032a000b0182000109d880060192000209d880023
:1032b000101a2000309d8800c01a2000409d880010
:1032c000801b2000509d8800401c2000609d8800cd
:1032d000001d2000709d8800d01d2000809d88006a
:1032e000a01e2000909d8800701f2000a09d8800d7
:1032f00050202000b09d880030212000c09d880013
:1033000020222000d09d880010232000e09d88000e
:1033100000242000f09d880000252000009e8800e9
:1033200000262000109e880010272000209e880084
:1033300020282000309e880030292000409e8800f0
:10334000502a2000509e8800802b2000609e88001c
:10335000b02c2000709e8800f02d2000809e8800f8
:10336000302f2000909e880070302000a09e8800a2
:10337000c0312000b09e880020332000c09e88000d
:1033800090342000d09e880000362000e09e880007
:1033900070372000f09e880000392000009f8800d0
:1033a000803a2000109f8800203c2000209f880049
:1033b000c03d2000309f8800703f2000409f880063
:1033c00030412000509f880000432000609f88000b
:1033d000d0442000709f8800b0462000809f880065
:1033e000a0482000909f8800a04a2000a09f88004d
:1033f000b04c2000b09f8800c04e2000c09f8800c5
:10340000f0502000d09f880020532000e09f8800cb
:1034100060552000f09f8800c057200000a0880061
:10342000205a200010a08800a05c200020a0880066
:10343000205f200030a08800c061200040a08800ec
:103440006064200050a088002067200060a08800f1
:10345000006a200070a08800e06c200080a0880036
:10346000e06f200090a08800e0722000a0a08800fb
:1034700010762000b0a0880040792000c0a088000d
:10348000907c2000d0a08800f07f2000e0a0880081
:10349000000006001e33ef0040062000009988005f
:1034a000800d200010998800c00d20002099880010
:1034b000000e200030998800400e200040998800be
:1034c000800e200050998800c00e2000609988006e
:1034d000100f200070998800500f200080998800fc
:1034e000a00f200090998800e00f2000a09988008c
:1034f00030102000b099880070102000c09988001a
:10350000c0102000d099880010112000e099880098
:1035100060112000f0998800b0112000009a880006
:1035200000122000109a880050122000209a880073
:10353000b0122000309a880000132000409a8800c2
:1035400060132000509a8800b0132000609a880011
:1035500010142000709a880070142000809a88004f
:10356000d0142000909a880030152000a09a88007e
:1035700090152000b09a8800f0152000c09a8800ad
:1035800060162000d09a8800c0162000e09a8800bb
:1035900030172000f09a8800a0172000009b8800b8
:1035a00000182000109b880070182000209b8800c5
:1035b000e0182000309b880060192000409b8800a4
:1035c000d0192000509b8800501a2000609b880072
:1035d000c01a2000709b8800401b2000809b880040
:1035e000c01b2000909b8800401c2000a09b8800ee
:1035f000c01c2000b09b8800401d2000c09b88009c
:10360000d01d2000d09b8800601e2000e09b880019
:10361000e01e2000f09b8800701f2000009c8800a6
:1036200010202000109c8800a0202000209c8800f2
:1036300030212000309c8800d0212000409c880050
:1036400070222000509c880010232000609c88007d
:10365000b0232000709c880050242000809c8800ab
:1036600000252000909c8800b0252000a09c8800a8
:1036700060262000b09c880010272000c09c880095
:10368000c0272000d09c880080282000e09c880073
:1036900030292000f09c8800f0292000009d88003f
:1036a000c02a2000109d8800802b2000209d8800cb
:1036b000502c2000309d8800102d2000409d880057
:1036c000f02d2000509d8800c02e2000609d8800b5
:1036d000902f2000709d880070302000809d880011
:1036e00050312000909d880040322000a09d88002d
:1036f00020332000b09d880010342000c09d880039
:1037000000352000d09d880000362000e09d880014
:10371000f0362000f09d8800f0372000009e8800e1
:1037200000392000109e8800003a2000209e88006a
:10373000103b2000309e8800203c2000409e8800e6
:10374000403d2000509e8800503e2000609e880032
:10375000703f2000709e8800a0402000809e88005e
:10376000d0412000909e880000432000a09e880049
:1037700030442000b09e880070452000c09e880024
:10378000b0462000d09e880000482000e09e8800bf
:1037900050492000f09e8800a04a2000009f880029
:1037a000004c2000109f8800604d2000209f880062
:1037b000c04e2000309f880030502000409f88007d
:1037c000a0512000509f880020532000609f880057
:1037d000a0542000709f880030562000809f8800f1
:1037e000c0572000909f880050592000a09f88005b
:1037f000f05a2000b09f8800a05c2000c09f880085
:10380000405e2000d09f880000602000e09f88007c
:10381000c0612000f09f88008063200000a0880025
:103820005065200010a088002067200020a088009c
:103830000069200030a08800f06a200040a08800c5
:10384000e06c200050a08800d06e200060a08800ae
:10385000e070200070a08800e072200080a0880046
:103860000075200090a0880020772000a0a088008c
:1038700040792000b0a08800807b2000c0a0880094
:10388000b07d2000d0a08800f07f2000e0a088005c
:0838900000000600ffff3700f5
:020000040000fa
:10389800ce1100000400000080000000d2110000da
:1038a8001400000080000000e6110000180000006d
:1038b80080000000fe1100002000000080000000d1
:1038c8001e12000000020000800000001e1400000c
:0c38d80000010000800000000000000063
:00000001FF
